:100000000C9446000C9463000C9463000C94630001
:100010000C9463000C9463000C9463000C946300D4
:100020000C9463000C9463000C9463000C946300C4
:100030000C9463000C9463000C9463000C940F0107
:100040000C9463000C9463000C9463000C946300A4
:100050000C9463000C9463000C9463000C94630094
:100060000C9463000C9463000C9463000C94630084
:100070000C9463000C9463000C9463000C94630074
:100080000C9463000C9463000C94630011241FBE55
:10009000CFEFD0E1DEBFCDBF11E0A0E0B1E0E4E3FF
:1000A000FDE000E00BBF02C007900D92A834B1073D
:1000B000D9F712E0A8E4B1E001C01D92AA3AB10755
:1000C000E1F70C94BF000C9400009C0112BE10924A
:1000D000A3011092A2018091A2019091A301821725
:1000E0009307C9F7089513BE86B7836086BF87B7A5
:1000F000836087BF8DE083BF12BE8DE781BF089507
:10010000882321F45D9BFECF6CB90895813039F4CA
:10011000EBE9F0E0808185FFFDCF60939C000895BE
:10012000682F80E00E94800080E090E00895CF93E7
:10013000DF9380E092E00E941E03C0E0D1E0CE0198
:100140000E94520580919802909199020E945D024E
:1001500080E094E00E941E03F2CFCF93DF93C8E0CB
:10016000D1E0CE010E9452058091980290919902AF
:100170000E945D0280E094E00E941E03F2CFCFEF68
:10018000D0E1DEBFCDBF0E9473001092900087E6E1
:1001900089B988E08AB901E02AE040E550E060E5ED
:1001A00070E084E00E943E0490939902809398024C
:1001B000789460E070E080E990E00E94020580E1C0
:1001C00091E00E94520500E010E02AE040E550E096
:1001D00062E571E08DEA90E00E94F0039093510196
:1001E0008093500186E291E00E9452052AE040E5AA
:1001F00050E064E472E087E990E00E94F00390939D
:100200009502809394020CE311E0C8010E9452050C
:1002100080919802909199020E948902F6CF1F92D4
:100220000F920FB60F9211242F933F934F935F932A
:100230006F937F938F939F93AF93BF93EF93FF93AE
:100240008091A2019091A30101969093A3018093C4
:10025000A2010E94CC02FF91EF91BF91AF919F91BB
:100260008F917F916F915F914F913F912F910F905F
:100270000FBE0F901F901895CF93DF93DC01C091B4
:100280004A01D0914B012097A1F1C817D90759F520
:1002900003C0AE17BF0741F52D913C911197211571
:1002A000310531F0FD0182819381F90193838283CD
:1002B000FD01228133812115310531F08D919C9111
:1002C0001197F90191838083CA17DB0731F48A8182
:1002D0009B8190934B0180934A01FD01138212820E
:1002E0001D921C9206C0FE010280F381E02D309722
:1002F00081F6DF91CF910895CF93DF93DC01409198
:100300004801509149014115510591F1481759078C
:1003100011F0FA0129C060E070E004C0A817B90725
:1003200011F5BF01ED01EC81FD81309741F080892D
:10033000918928893989820F931F918B808B4A1765
:100340005B0739F4FD018481958190934901809385
:1003500048016115710561F0ED018C819D81FB0102
:100360009583848305C0FC01848195810097B1F653
:10037000DF91CF910895CF93DF93EC01A0914A01D3
:10038000B0914B01109789F12A85FD018285821772
:1003900080F48D919C9111970097D1F4D0934B01EB
:1003A000C0934A01BB83AA8319821882CD93DC9340
:1003B00024C0FD0182819381009711F0DC01E5CF1B
:1003C000FD01D383C2831B821A82B983A88315C01F
:1003D00099838883ED91FC911197D383C283119601
:1003E000DC93CE93BB83AA8308C090934B01809388
:1003F0004A011B821A8219821882DF91CF910895D7
:10040000E0919E02F0919F02029697838683089561
:100410001F93CF93DF938FB7182F1078F894E09144
:100420009C02F0919D0285858370833019F4CF0181
:100430000E94BB01A0914A01B0914B01109789F035
:10044000ED01EA81FB81F0934B01E0934A01309783
:1004500011F011821082FD011382128211961C92FA
:100460001E92E0919C02F0919D02AE17BF0731F4FD
:10047000848583878FB7812B8FBF1BC0F0939F022A
:10048000E0939E02B0939D02A0939C028485838793
:10049000E0919C02F0919D0284858387E0919C020B
:1004A000F0919D02868197810E94AB048FB7812BCA
:1004B0008FBFDF91CF911F9108951F93CF93DF934B
:1004C000EC0180919C0290919D028C179D07E9F0B0
:1004D0001FB7F894CE010E943C01CE010E947C011E
:1004E0008D8582608D87CE010E94BB019A85E09147
:1004F0009C02F0919D028285891710F40E940802E7
:100500009FB7812F8078892B8FBFDF91CF911F916B
:100510000895FF920F931F938C01FFB6F8940E94E9
:100520003C01C8010E947C01F80185858D7F85878B
:1005300080919C0290919D020817190711F40E9466
:1005400008029FB78F2D8078892B8FBF1F910F9145
:10055000FF900895FF920F931F938C01FFB6F894BC
:100560000E943C01C8010E947C01F801158680911F
:100570009C0290919D020817190711F40E9408022D
:100580009FB78F2D8078892B8FBF1F910F91FF9080
:1005900008950E940802FDCF1F93CF93DF93C0916F
:1005A0004801D0914901209789F18889998901975B
:1005B000998B888B892B51F510E08D8582608D8712
:1005C000CE010E94BB01E0919C02F0919D029A85B0
:1005D0008285891708F411E0EC81FD811D821C825F
:1005E000309779F080899189892B11F4EF01E5CF5B
:1005F000F0934901E0934801112341F00E94080261
:1006000019C01092490110924801F6CF80919A02C8
:10061000882381F0E0919C02F0919D0283858150B6
:100620008387E0919C02F0919D028385882311F4D9
:100630000E940802DF91CF911F9108951F93CF93DD
:10064000DF939C018FB7182F1078F894E0919C02EB
:10065000F0919D0285858D7F8587A0914801B0919D
:100660004901109719F0C0E0D0E017C0E0919C025A
:10067000F0919D02F0934901E093480115821482A4
:10068000E0919C02F0919D02318B208B0E94080228
:100690008FB7812B8FBF4FC0DC01FD01808991890D
:1006A0002817390738F5821B930B918B808BE091CB
:1006B0009C02F0919D02B583A483E0919C02F0918D
:1006C0009D02318B208B209739F080919C02909174
:1006D0009D029D838C8308C080919C0290919D0215
:1006E00090934901809348010E9408028FB7812BA3
:1006F0008FBF21C0FD0180899189281B390B84811E
:100700009581ED01009741F680919C0290919D02A8
:100710009D838C83E0919C02F0919D02158214824E
:10072000E0919C02F0919D02318B208B0E94080287
:100730008FB7812B8FBFDF91CF911F910895AF921B
:10074000BF92CF92DF92EF92FF920F93CF93DF93FE
:10075000EC015B01CA016901452B29F48DB79EB7F5
:10076000821B930B029799878887DF86CE86A60126
:1007700069E970E00E94FB04E885F985EC0DFD1D38
:100780003197A08231978B2D992780833197FF83F2
:10079000EE8380E0813049F4EE81FF818FB7808362
:1007A0003197FF83EE8382E0F5CFEE81FF811082E7
:1007B0003197FF83EE838F5F813260F30A8785E094
:1007C0008C878B8783E08D87FB8AEA8ADF91CF91C4
:1007D0000F91FF90EF90DF90CF90BF90AF90089572
:1007E000EF92FF920F931F93CF93DF93DC01780179
:1007F0008FB7182F1078F894E0919B02EE23C9F080
:1008000080910102882371F4F0E081E092E0EC0134
:100810002D9703C08D85882341F481E08D87EF17E4
:1008200071F407C0F0E0C4EFD1E0FF5F6496EF170A
:1008300089F78FB7812B8FBFC0E0D0E017C0022FA0
:100840009A01AB01BD01CE010E949F03CE010E941F
:10085000BB01E0919C02F0919D0292858A859817D8
:1008600010F40E9408028FB7812B8FBFCE01DF9159
:10087000CF911F910F91FF90EF900895DF92EF922B
:10088000FF920F931F93CF93DF93382FEB01E22E4C
:10089000F02EDFB6F89480939B028823B1F020E01D
:1008A00064EF71E0E22FFF27EE0FFF1FEE0FFF1F37
:1008B000CF01880F991F880F991FE80FF91FE60FC6
:1008C000F71F15862F5F321769F710924B011092B0
:1008D0004A0100E010E020E064EA71E089EC92E077
:1008E0000E94F00390934D0180934C010E943C01C3
:1008F000F0929A0210924901109248012E2DAE01F9
:1009000060E070E080E090E00E94F00390934F017F
:1009100080934E0190939F0280939E02E0914C0140
:10092000F0914D01F0939D02E0939C0286819781A6
:100930000E94AB049FB78D2D8078892B8FBF80914B
:100940004E0190914F01DF91CF911F910F91FF9038
:10095000EF90DF900895F8940F920FB60F921F92C8
:100960002F923F924F925F926F927F928F929F92BF
:10097000AF92BF92CF92DF92EF92FF920F931F93AD
:100980002F933F934F935F936F937F938F939F9397
:10099000AF93BF93CF93DF93EF93FF938F939F9387
:1009A0008DB79EB70E9400029F918F918DBF9EBF11
:1009B000FF91EF91DF91CF91BF91AF919F918F9177
:1009C0007F916F915F914F913F912F911F910F9167
:1009D000FF90EF90DF90CF90BF90AF909F908F905F
:1009E0007F906F905F904F903F902F901F900F904F
:1009F0000FBE0F901895DC0101C06D93415050401F
:100A0000E0F70895EF92FF920F931F93CF93DF9338
:100A10008C017B01892B11F4672BD1F16EE070E022
:100A200081E090E00E948505FC01009789F1DC01DE
:100A300080E88383E114F10471F0F386E28681E8B3
:100A400083838091A0029091A102892B21F4F093DD
:100A5000A102E093A00201151105E1F011870087C2
:100A60008381826083838091A2029091A302892B6B
:100A700089F4F093A302E093A2028091A4029091E2
:100A8000A502892B39F4F093A502E093A40202C0D9
:100A9000A0E0B0E0CD01DF91CF911F910F91FF90C9
:100AA000EF9008950F931F93CF93DF938C01E09104
:100AB000A202F091A302838181FF1FC0C0E0D0E0B9
:100AC0000AC0FD0120853185BD01F9010995892BF9
:100AD00011F0CFEFDFEFF80181918F01A091A20219
:100AE000B091A302882369F7FD0120853185BD01FE
:100AF0008AE0F9010995892B11F0CFEFDFEFCE01E4
:100B0000DF91CF911F910F9108950F931F93CF9372
:100B1000DF93869F8001879F100D969F100D1124F3
:100B2000C8010E94A105EC01009729F0A80160E02E
:100B300070E00E94FB04CE01DF91CF911F910F91D5
:100B40000895CF93DF93AC01029710F442E050E098
:100B5000A091A802B091A902FD01C0E0D0E020E080
:100B600030E020C0808191818417950769F48281EB
:100B70009381209719F09B838A8304C09093A902E4
:100B80008093A802CF0132C04817590738F42115C5
:100B9000310519F08217930708F49C01EF010280D8
:100BA000F381E02D3097F1F62115310589F1C90166
:100BB000841B950B049708F4A901E0E0F0E026C03F
:100BC0008D919C91119782179307E9F44817590763
:100BD00079F4ED018A819B81309719F093838283A8
:100BE00004C09093A9028093A802CD01029649C047
:100BF000841B950BFD01E80FF91F41935193029758
:100C00008D939C933AC0FD01A281B3811097C1F6E8
:100C10008091A6029091A702892B41F48091430113
:100C2000909144019093A7028093A60220914501E0
:100C3000309146012115310541F42DB73EB7809121
:100C4000410190914201281B390BE091A602F091DD
:100C5000A7022E1B3F0B2417350788F0CA01029606
:100C60002817390760F0CF01840F951F02969093E3
:100C7000A7028093A60241935193CF0102C080E066
:100C800090E0DF91CF910895CF93DF93009709F41F
:100C90004EC0EC0122971B821A82A091A802B0914B
:100CA000A902109711F140E050E001C0DC01AC173F
:100CB000BD0700F1BB83AA83FE0121913191E20FB0
:100CC000F31FEA17FB0771F42E5F3F4F8D919C9144
:100CD0001197820F931F99838883FD0182819381ED
:100CE0009B838A834115510559F4D093A902C0937F
:100CF000A8021DC0FD0182819381AD010097B1F66C
:100D0000FA01D383C28321913191E20FF31FEC17D3
:100D1000FD0769F42E5F3F4F88819981820F931FF1
:100D2000FA01918380838A819B8193838283DF91FF
:040D3000CF910895C2
:100D3400746872656164320074687265616431005C
:100D44006372656174696E6720746872656164209A
:100D540031202E2E2E006372656174696E672074D3
:100D640068726561642032202E2E2E006D61696EDA
:080D7400002000AA02000000AB
:00000001FF
